S024000062696E2F6F70656E626C745F6F6C696D65785F73746D3332683130332E73726563A3
S315080000005C090020AD260008912600089126000804
S3150800001091260008912600089126000891260008D6
S3150800002091260008912600089126000891260008C6
S3150800003091260008912600089126000891260008B6
S3150800004091260008912600089126000891260008A6
S315080000509126000891260008912600089126000896
S315080000609126000891260008912600089126000886
S315080000709126000891260008912600089126000876
S315080000809126000891260008912600089126000866
S315080000909126000891260008912600089126000856
S315080000A09126000891260008912600089126000846
S315080000B09126000891260008912600089126000836
S315080000C09126000891260008912600089126000826
S315080000D09126000891260008912600089126000816
S315080000E09126000891260008912600089126000806
S315080000F091260008912600089126000891260008F6
S3150800010091260008912600089126000891260008E5
S3150800011091260008912600089126000891260008D5
S3150800012091260008912600089126000891260008C5
S3150800013091260008912600089126000891260008B5
S3150800014091260008912600089126000891260008A5
S3150800015040F2F003C2F200031B78CBB94FF4805388
S31508000160C4F202039A6942F010029A614FF480536E
S31508000170C4F201035A6822F470425A605A6842F47B
S31508000180E0425A6040F2F003C2F2000301221A70FC
S3150800019001284FF48053C4F201034FF400620CBFE8
S315080001A05A611A61704700BF4FF40063C4F2010335
S315080001B0986800F00100704700B583B000230093EB
S315080001C001934FF48053C4F202031A6842F0010205
S315080001D01A6059680022CFF6FF020A405A601A6868
S315080001E022F0847222F480321A601A6822F480227D
S315080001F01A605A6822F4FE025A604FF41F029A6087
S315080002001A6842F480321A604FF48053C4F202032B
S3150800021040F2DC52196801F400310191009901316C
S315080002200091019911B900999142F3D14FF4805385
S31508000230C4F202031B6813F4003F06D142F21070A1
S31508000240C0F60000672101F0D5FC4FF40053C4F254
S3150800025002031A6842F010021A601A6822F00302B2
S315080002601A601A6842F002021A604FF48053C4F208
S3150800027002035A685A605A6842F400525A605A6829
S3150800028042F480625A605A6822F47C125A605A68AC
S3150800029042F4E8125A601A6842F080721A604FF403
S315080002A08053C4F202031A6812F0007FFBD04FF4A1
S315080002B08053C4F202035A6822F003025A605A684D
S315080002C042F002025A604FF48053C4F202035A689D
S315080002D002F00C02082AFAD14FF48053C4F2020342
S315080002E09A6942F004029A614FF40062C4F201026C
S315080002F0116821F00F011160116841F004011160C5
S315080003005A6822F480025A60DA6942F40002DA6115
S3150800031001F0E4F901F0F0F9FCE700BF08B501F0D7
S315080003202BFE08BD08B501F083FE08BD08B540F2EE
S31508000330F403C2F200031B68052B01D101F01CFE71
S3150800034008BD00BF40F23073C2F200039B7A2BB19E
S3150800035040F2F403C2F2000305221A60704700BF98
S3150800036040F2F403C2F2000304221A60704700BF89
S31508000370704700BF704700BF10B5062810D140F27D
S315080003805073C2F200031B681A7802F07F02012A32
S3150800039008D15A7942B99A78212A07D0022010BD85
S315080003A0022010BD022010BD022010BD40F2FD4201
S315080003B0C0F600029A6100245C82204600F09EF88E
S315080003C0204610BD0220704721B9002814BF02201C
S315080003D0002070470220704710B501F059FE40F220
S315080003E05073C2F200031B6800249C7200F0E4F804
S315080003F001F04EF940F2F403C2F200031C6010BD8E
S3150800040010B540F25073C2F200031B6800249C72B8
S3150800041042F25872C0F60002D2795A72DC7220464D
S3150800042000F0F8FF20464FF4007100F0FDFF20466B
S31508000430102101F005F82046402101F0A7F82046D2
S31508000440802101F091F8204601F056F840F20803A1
S31508000450C2F20003204693F82C1001F0DBF8204680
S3150800046001F038F80120214600F0DEFF01204FF4A4
S31508000470807101F079F80120C02101F087F8012088
S31508000480402101F0B7F80120402101F0C3F801200E
S315080004904FF4405100F0F0FF0120202100F0D0FF7A
S315080004A0204600F09BFD40F2F403C2F2000301224D
S315080004B01A6010BD08B540F26401C2F2000100F0EE
S315080004C0DFFA08BD08B540F20001C2F2000100F0EB
S315080004D0D7FA08BD08B540F25073C2F200031B688C
S315080004E0D978052908D840F26C03C2F2000303EB59
S315080004F0C10100F0C5FA08BD002008BD08B540F2E4
S315080005005C01C2F2000100F0BBFA08BD08B545F669
S315080005104443C4F200031A6892B240F21C73C2F252
S3150800052000031A801A8840F25473C2F200031B882B
S31508000530134003F400739BB283B145F64443C4F2F7
S3150800054000034FF6FF521A6040F2F103C2F20003AD
S315080005501A780132D2B21A70FFF7E8FE40F21C731D
S31508000560C2F200031A8840F25473C2F200031B88D1
S31508000570134003F400439BB20BB100F0B3FD40F205
S315080005801C73C2F200031A8840F25473C2F20003C5
S315080005901B88134003F480639BB263B145F644435A
S315080005A0C4F200034FF6FF321A6040F20803C2F2A3
S315080005B000035B68984708BD08B50120FFF7C8FD2A
S315080005C045F64043C4F2000301221A6040F2547211
S315080005D0C2F200020020186045F64441C4F2000148
S315080005E008604FF4E0511180196008BD08B538B9A4
S315080005F040F25073C2F200031B6801221A8208BD3A
S3150800060040F24C73C2F200031B681B68984740F21D
S315080006105073C2F2000318680A3008BD08B538B925
S3150800062040F25073C2F200031B6801221A8208BD09
S3150800063040F24C73C2F200031B689B68984740F26D
S315080006405073C2F2000318680C3008BD08B538B9F3
S3150800065040F25073C2F200031B6802221A8208BDD8
S3150800066040F22073C2F2000300221A8040F250734F
S31508000670C2F200031A68137813F07F0317D1537A6E
S3150800068013F0200F1FBF40F22072C2F200020221AF
S31508000690117013F0400F40F22073C2F200031A786B
S315080006A014BF42F0010222F001021A702BE0012B5E
S315080006B035D0022B38D1537903F00F0213F0800F8F
S315080006C010D0920002F1804202F5B842136803F096
S315080006D03003102B17D140F22073C2F20003012217
S315080006E01A7010E0920002F1804202F5B8421368CF
S315080006F003F44053B3F5805F01BF40F22073C2F2A2
S31508000700000301221A7040F24C73C2F200031B6800
S315080007101B69984740F22070C2F2000008BD40F2FB
S315080007202070C2F2000008BD002008BDF8B540F2EE
S315080007305073C2F200031C68238A227A002B08BF72
S31508000740042A29D140F2F803C2F200031B78012BD0
S315080007501AD145F65043C4F200031A6892B243F21E
S315080007600203C2F2000313445B0000221A6040F23F
S315080007705873C2F200033021198040F2F803C2F21E
S3150800078000031A70042632E040F25873C2F20003DE
S3150800079010221A8007262AE0A58AAB428CBF0226B9
S315080007A004269D4228BF1D46A36928469847074642
S315080007B0002000F0FFFE014638462A4600F000FEFB
S315080007C00020294600F016FF238A5B1B2382638AD2
S315080007D01D44658240F25873C2F2000330221A8023
S315080007E040F25673C2F200034FF440521A8040F2A8
S315080007F05073C2F200031B681E72F8BD08B540F2BA
S315080008005073C2F200031A68D17840F29403C2F218
S3150800081000035B788B420DD393786BB993886BB9D9
S31508000820917240F24C73C2F200031B685B689847EA
S31508000830002008BD022008BD022008BD022008BD10
S3150800084010B540F25074C2F20004226840F22873D0
S31508000850C2F200031B689B695079D17898472368D0
S315080008609A7A92B198B91A799AB99B789BB940F253
S315080008704C73C2F200031B68DB68984723685A79F1
S31508000880DA72DA781A73002010BD022010BD022031
S3150800089010BD022010BD022010BD00BF10B540F2E9
S315080008A05073C2F200031A68137813F07F0305D158
S315080008B0537A23F020035372002010BD022B6FD108
S315080008C05388002B6ED11379002B6DD1517921F005
S315080008D0800011F0800F4FEA800303F1804303F58F
S315080008E0B84319BF1C6804F030041B6803F440546D
S315080008F040F29403C2F200031B78984256D2002CA9
S3150800090056D0937A002B55D011F0800F12D0830061
S3150800091003F1804303F5B8431B6803F03003102B3B
S3150800092035D1C4B2204600F00BFE2046302100F037
S3150800093087FD2CE0840004F1804404F5B84423685C
S3150800094003F44053B3F5805F21D198B940F2080308
S31508000950C2F2000393F82C1000F05CFE22684BF6F6
S315080009608F73134083F4405343F4004343F08003EA
S3150800097023600CE000F0D0FD22684BF68F7313401D
S3150800098083F4405343F4004343F08003236040F26A
S315080009904C73C2F200031B685B699847002010BDC0
S315080009A0022010BD022010BD022010BD022010BD7D
S315080009B0022010BD022010BD10B540F25073C2F2DD
S315080009C000031868427922F0800112F0800F4FEA7E
S315080009D0810303F1804303F5B84319BF1C6804F08B
S315080009E030041B6803F4405440F29403C2F2000337
S315080009F01B78994227D243883BBB44B3837A43B3D7
S31508000A0012F0800F4FEA810202F1804202F5B842E5
S31508000A1011681DBF48F6BF730B4083F010034BF6F1
S31508000A208F7304BF0B4083F4805343F4004343F0B1
S31508000A308003136040F24C73C2F200031B689B6983
S31508000A409847002010BD022010BD022010BD0220CC
S31508000A5010BD022010BD00BF08B540F25073C2F2A7
S31508000A6000031B685A7A42F020025A7240F24C730D
S31508000A70C2F200031B68DB699847002008BD00BF67
S31508000A8040F25073C2F200031B685A8A18B9898863
S31508000A908A1A1A82704708681044704708B540F2E7
S31508000AA00803C2F20003002093F82C1000F0B2FDF0
S31508000AB040F25073C2F200031B68187A08280CD15A
S31508000AC040F25673C2F200034FF480521A8040F285
S31508000AD05873C2F2000310221A80092814BF002096
S31508000AE0012008BD70B582B045F65043C4F2000334
S31508000AF01A6892B243F20403C2F2000313445B007D
S31508000B001D6840F25073C2F200031B681A7A092A5C
S31508000B101BD0ADB26D0005F1804505F5C0452A78B4
S31508000B201A7040F25074C2F2000423686A785A7048
S31508000B302668A88800F0A6FD70802668288900F037
S31508000B40A1FDB080AA892368DA8040F25073C2F208
S31508000B5000031B6801221A72DA88002A77D15C78AA
S31508000B601A7812F07F022ED1092C02D1FFF746FE21
S31508000B703BE0052C0FD193F90320002AB8BF0822C1
S31508000B805EDB9A78002A55D19A88002A54D19B7A36
S31508000B90002B39D052E0032C07D1DA78012A25D167
S31508000BA09B881BBBFFF758FF1FE0012C1ED1DA7884
S31508000BB0012A1BD19A88CAB95B7A13F0200F15D07F
S31508000BC0FFF76CFE11E0012A04D10B2C0ED1FFF7BA
S31508000BD037FE0AE0022A09D1012C02D1FFF75EFE90
S31508000BE003E0032C02D1FFF7E7FE68B140F2287351
S31508000BF0C2F200031B685B6920469847032808BFB2
S31508000C0009221DD00822D8B945F65043C4F200037C
S31508000C101A6892B243F20203C2F2000313445B005D
S31508000C2000221A6040F25873C2F2000330221A807A
S31508000C30062205E0082203E0082201E00822FFE771
S31508000C4040F25073C2F200031B681A7217E15A7811
S31508000C50062A21D11A7812F07F0F40F0A9809B78D6
S31508000C60012B06D140F22873C2F200031B68DA6929
S31508000C708DE0022B06D140F22873C2F200031B68EE
S31508000C801A6A84E0032B40F0938040F22873C2F27C
S31508000C9000031B685A6A7AE0002A52D15A88002A49
S31508000CA040F086805A6822F47F42B2F5003F7FD131
S31508000CB01A7812F07F0204D19B88002B00F0E2809C
S31508000CC076E0012A14D140F22872C2F200021268B4
S31508000CD09269587900219047002869D140F25073EB
S31508000CE0C2F200031B689B7A002B40F0D0805FE0BD
S31508000CF0022A5DD15A7902F00F0112F0800F4FEAED
S31508000D00810303F1804303F5B84319BF186800F05F
S31508000D1030001B6803F4405040F29403C2F200030B
S31508000D201B78994244D212F0700F14BF0023012396
S31508000D3000280CBF002003F00100002840F0AC801A
S31508000D4036E0082A05D11B7813F07F0F00F0A9803A
S31508000D502EE00A2A2CD11A7802F07F02012A27D11E
S31508000D609A7A2AB35A881ABB5A6822F47F42B2F58D
S31508000D70803F1DD140F22872C2F2000212689269C1
S31508000D80587900219047002800F0908010E07AB149
S31508000D9040F25074C2F200042368002058829A6117
S31508000DA0904723681A8A4FF6FF718A4226D120E0B7
S31508000DB040F22873C2F20003196840F25073C2F277
S31508000DC000031A680B6950789847032807D140F240
S31508000DD05073C2F200031B6809221A724FE040F2F0
S31508000DE05073C2F200031B681A8A4FF6FF718A42D3
S31508000DF002D109221A7242E0022800D012B908224A
S31508000E001A723CE093F9001000292FDAD98801916B
S31508000E100198824202D9019A1A821CE091421AD993
S31508000E2040F22871C2F20001096891F82C1091422B
S31508000E3006D940F2F802C2F20002002111700AE057
S31508000E4092FBF1F001FB10222AB940F2F802C2F235
S31508000E5000020121117040F22872C2F200021268E3
S31508000E6092F82C209A82FFF761FC08E003221A7296
S31508000E7040F25673C2F200034FF440521A80FFF74D
S31508000E800DFE18E040F24D62C0F6000280E740F21F
S31508000E904D62C0F600027BE740F24D62C0F60002E2
S31508000EA076E740F2ED52C0F6000271E740F21D62A5
S31508000EB0C0F600026CE702B070BD00BF70B540F224
S31508000EC05073C2F200031C68237A022B18BF042B46
S31508000ED008BF082274D0032B18BF052B63D1228ABA
S31508000EE0A369ABB1A2B1A58A954228BF1546284683
S31508000EF098470646238A5B1B2382638A2B446382B0
S31508000F00002000F067FB014630462A4600F072FAD8
S31508000F10238A002B5DD040F25673C2F200034FF4C9
S31508000F2040521A800020014600F064FB40F25873D4
S31508000F30C2F2000330221A80238AA28A9A4207D86C
S31508000F4040F25073C2F200031B6803221A7223E0B0
S31508000F503BB140F25073C2F200031B6805221A72B5
S31508000F601AE040F25073C2F200031B6806221A7296
S31508000F7045F65043C4F200031A6892B243F20203DC
S31508000F80C2F2000313445B0000221A6040F2587351
S31508000F90C2F2000330221A8040F25073C2F20003F4
S31508000FA01B681A7A0CE0072B18BF082208D140F2F2
S31508000FB02873C2F200031B68DB6898470822FFE71C
S31508000FC040F25073C2F200031B681A72FFF766FDFF
S31508000FD070BDA38A002BC4D1B2E700BF70B440F23B
S31508000FE09403C2F200031D789DB1002340F60F76E4
S31508000FF0DAB2910001F1804101F5B8410C6842F47A
S31508001000004242F08002344022430A6001339D4286
S31508001010EED840F0800045F64C43C4F20003186051
S3150800102070BC704708B540F25073C2F200031A68E4
S31508001030137A022B18BF042B08D1FFF777FB40F26F
S315080010405073C2F200031B681A7A1DE0062B18BFFC
S31508001050082219D15378052B0DD1137813F07F0F79
S3150800106009D1D078FFF7BAFF40F24C73C2F20003F9
S315080010701B681B6A984740F22873C2F200031B6874
S315080010809B6898470822FFE740F25073C2F20003B4
S315080010901B681A72FFF702FD08BD00BF704700BF44
S315080010A008B540F25072C2F2000240F23073C2F242
S315080010B00003136002221A7240F22872C2F200027A
S315080010C040F20803C2F20003136040F24C72C2F207
S315080010D0000240F23801C2F2000111601B6898470D
S315080010E008BD00BF2DE9F04383B00023ADF80630F4
S315080010F045F64447C4F2000740F21C74C2F20004E5
S3150800110040F22C76C2F2000640F2B408C2F2000899
S3150800111040F2D009C2F2000940F25675C2F2000543
S3150800112043E1238803F00F033370002B40F00F814F
S315080011304FF4B843C4F200031A6892B22A80298889
S3150800114001F0300140F25872C2F2000211802A887A
S3150800115002F440522A8019684BF6BF720A4082F49C
S31508001160005282F0200242F4004242F080021A60E5
S31508001170238803F010039BB2002B46D14FF4B844E2
S31508001180C4F20004226848F60F7313402360FFF781
S3150800119049FF22684BF6BF73134040F25672C2F2FB
S315080011A00002128802F4805292B20AB183F4805384
S315080011B040F25672C2F20002128802F4005292B24B
S315080011C00AB183F4005340F25872C2F20002128840
S315080011D002F0100292B20AB183F0100340F258727C
S315080011E0C2F20002128802F0200292B20AB183F01B
S315080011F0200348F28002CFF6FF721A4392B24FF4E8
S31508001200B843C4F200031A60D6E04FF4B843C4F2F8
S3150800121000031B689BB2ADF80630BDF8063003F430
S3150800122000639BB2002B46D04FF4B844C4F20004C6
S31508001230226840F68F7313402360FFF753FC226839
S315080012404BF6BF73134040F25672C2F20002128880
S3150800125002F4805292B20AB183F4805340F2567275
S31508001260C2F20002128802F4005292B20AB183F462
S31508001270005340F25872C2F20002128802F01002BD
S3150800128092B20AB183F0100340F25872C2F2000219
S31508001290128802F0200292B20AB183F0200348F2C3
S315080012A08002CFF6FF721A4392B24FF4B843C4F2E3
S315080012B000031A6080E0BDF806301BB2002B74DA12
S315080012C04FF4B844C4F20004226840F68F73134002
S315080012D02360FFF7F3FD22684BF6BF73134040F215
S315080012E05672C2F20002128802F4805292B20AB111
S315080012F083F4805340F25672C2F20002128802F456
S31508001300005292B20AB183F4005340F25872C2F204
S315080013100002128802F0100292B20AB183F010039A
S3150800132040F25872C2F20002128802F0200292B20B
S315080013300AB183F0200348F28002CFF6FF721A43FF
S3150800134092B24FF4B843C4F200031A6034E09B002B
S3150800135003F1804303F5B8431A6892B2ADF8062044
S31508001360BDF8062012B2002A09DA196840F68F720B
S315080013700A401A603378013B59F823309847BDF87C
S31508001380063003F080039BB27BB13278920002F1FB
S31508001390804202F5B842116848F60F730B40136095
S315080013A03378013B58F8233098473B689AB2228035
S315080013B013F4004F7FF4B5AE03B0BDE8F08300BF69
S315080013C010B4531C01F1005101F5405252005B1054
S315080013D00DD00432023010F8014C10F8021C41EA14
S315080013E0042122F8041C04320230013BF3D15DF8D3
S315080013F0044B7047013201F1005101F54051490093
S31508001400531005D051F8042B20F8022B013BF9D1D3
S31508001410704700BF4FF6F873034045F65042C4F2D2
S3150800142000021360704700BF800000F1804202F599
S31508001430B842106848F68F13034019431160704785
S31508001440800000F1804202F5B842106848F6BF7382
S31508001450034001F0100080B208B183F0100301F0D8
S31508001460200189B209B183F0200343F4004343F015
S3150800147080031360704700BF800000F1804202F5C8
S31508001480B84210684BF68F73034001F4805080B25F
S3150800149008B183F4805301F4005189B209B183F489
S315080014A0005343F4004343F080031360704700BFC2
S315080014B0800000F1804202F5B842116848F6BF7311
S315080014C00B4083F0300343F4004343F0800313607A
S315080014D0704700BF800000F1804202F5B8421168EB
S315080014E04BF68F730B4083F4405343F4004343F0A9
S315080014F080031360704700BF800000F1804202F548
S31508001500B842116840F60F630B4043F4004343F0BA
S3150800151080031360704700BF800000F1804303F525
S31508001520B8431A6812F4804F08D0196840F60F724B
S315080015300A4042F4404242F080021A60704700BFF7
S31508001540800000F1804303F5B8431A6812F0400F93
S3150800155008D0196840F60F720A4042F4004242F079
S31508001560C0021A60704700BF45F65043C4F2000334
S315080015701A684FF6FE730B4092B202EBC00000F1F8
S31508001580005202F5405252001360704745F6504328
S31508001590C4F200031B684FF6FE720A409BB203EBC7
S315080015A0C00043F20403C2F2000303445B001A605E
S315080015B0704700BF45F65043C4F200031B689BB250
S315080015C003EBC00000F1005303F540535B00188895
S315080015D0704700BF45F65043C4F200031B689BB230
S315080015E003EBC00043F20403C2F2000303445B00AA
S315080015F01888704745F65043C4F200031B689BB22F
S3150800160003EBC00043F20203C2F2000303445B008B
S315080016101960704745F65043C4F200031B689BB235
S3150800162003EBC00043F20603C2F2000303445B0067
S315080016303E290BD94A0911F01F0F04BF02F1FF32E8
S3150800164092B2920242F400421A6070474A0811F0B8
S31508001650010F1CBF013292B292021A60704700BF96
S3150800166045F65043C4F200031B689BB203EBC00067
S3150800167043F20603C2F2000303445B001868C0F392
S3150800168009007047C3B2000A40EA0320704700BF4A
S3150800169045F64443C4F200030020186040F2547330
S315080016A0C2F200034FF406421A8045F64043C4F2DC
S315080016B000031A60704700BF70B50E4600F07F053C
S315080016C02846FFF7CDFF04462846FFF783FF014665
S315080016D030462246FFF78EFE204670BD08B500F05C
S315080016E08DFA00F083FA00F011FD00F0F1FC00F02D
S315080016F00DF800F069FA08BD08B500F079FA00F0AF
S3150800170021FD00F00FF800F03FFA08BD08B500F01B
S315080017105DF800F037FB40F2EC03C2F20003022248
S315080017201A7008BD08B540F2FC00C2F2000000F0CD
S31508001730C3FB01280BD140F2EC03C2F200030222DC
S315080017401A7040F2FC00C2F2000000F05FF808BD13
S3150800175008B500F06DFB08BD08B540F2EC03C2F20F
S3150800176000031B78022B02D1C9B200F067FB00F018
S3150800177045F808BD40F2EC03C2F200031B78012BC2
S3150800178001D9032B01D1002070473F20704700BFC5
S3150800179040F2EC03C2F200031B78012B01D9032B9C
S315080017A001D1002070473F20704700BF08B500F000
S315080017B01BF808BD40F23C13C2F20003FE22DA70A1
S315080017C018710222A3F84420704700BF40F23C1368
S315080017D0C2F2000300221A709A6483F84220A3F822
S315080017E044209A705A70704740F23C13C2F20003C4
S315080017F01878003018BF0120704700BF40F23C132C
S31508001800C2F20003002283F84220704738B5044626
S315080018100178FF291ED140F23C14C2F200040023CD
S31508001820637001252570FF22E27010222271637110
S31508001830FFF7A0FFA071FFF7ABFFE071FFF7A8FF66
S31508001840000A20726572A5720823A4F8443000F0D5
S315080018503FFC79E140F23C13C2F200031B78012BEE
S3150800186040F09081C939352900F26B81DFE811F023
S31508001870DB00690169016501690169015901FC001B
S3150800188042012F016901690169016901690169015B
S3150800189069016901690169016901690169016901EA
S315080018A069016901690169016901690169016901DA
S315080018B069016901690169016901690169016901CA
S315080018C0690169017F0054003600730069016901E6
S315080018D06901A1006901B900BD00CE004578FFF78E
S315080018E049FF0138854203DD2220FFF763FF2BE11C
S315080018F040F23C15C2F20005281DA96C627800F07A
S315080019009FF9FF23EB706278AB6C1344AB64637882
S315080019100133A5F8443017E14578FFF72BFF013866
S31508001920854203DD2220FFF745FF0DE1616840F29D
S315080019303C15C2F20005A964281D627800F080F9FA
S31508001940FF23EB706278AB6C1344AB6463780133A6
S31508001950A5F84430F8E040F23C13C2F20003FF2237
S31508001960DA7042689A640122A3F84420ECE040F257
S315080019703C13C2F20003FF22DA709B6C406840B148
S315080019801844002213F8011B0A44D2B28342F9D143
S3150800199000E0002240F23C13C2F20003C3F807201D
S315080019A001221A7100225A719A710822A3F844205A
S315080019B0CAE040F23C13C2F20003FF22DA7042F298
S315080019C0C072C0F600029A6400221A715A719A719E
S315080019D00721D9711A725A729A720822A3F84420FA
S315080019E0B2E00020FFF7E6FEAEE040F23C13C2F29A
S315080019F00003FF22DA7000221A71597859719A7118
S31508001A00DA711A720622A3F844209DE040F23C13CC
S31508001A10C2F2000300221A705A70FF22DA700122FD
S31508001A20A3F8442090E040F23C13C2F200039D6CF8
S31508001A30FFF7A0FE411E2846621C00F04DFB18B9B0
S31508001A403120FFF7B7FE7FE040F23C14C2F20004F3
S31508001A50FF23E370A56CFFF78DFE013D2844A064C3
S31508001A600123A4F844306FE04578FFF783FE023877
S31508001A70854203DD2220FFF79DFE65E040F23C1318
S31508001A80C2F20003FF22DA700122A3F8442061782B
S31508001A9039B900F031FB002856D13120FFF78AFE0C
S31508001AA052E040F23C13C2F20003986CA21C00F00C
S31508001AB013FB18B93120FFF77DFE45E040F23C13D1
S31508001AC0C2F2000361789A6C0A449A643CE040F2D8
S31508001AD03C14C2F20004FF23E370002525716571EA
S31508001AE0FFF748FEA071E571257265720723A4F811
S31508001AF0443029E040F23C13C2F20003986C616856
S31508001B0000F0EEFA18B93120FFF754FE1CE040F257
S31508001B103C13C2F20003FF22DA700122A3F8442024
S31508001B2012E000F06FF840F23C13C2F20003FF2205
S31508001B30DA700122A3F8442006E03120FFF73AFEC6
S31508001B4002E02020FFF736FE40F23C13C2F2000303
S31508001B5093F84230012B02D11020FFF72BFE40F2FA
S31508001B603C13C2F20003B3F844100BB2002B09DD94
S31508001B7040F23C10C2F20000012380F842300330E4
S31508001B80FFF7EAFD38BD00BF08B5FFF70FFE0128CD
S31508001B9019D040F28813C2F200031B78012B12D128
S31508001BA000F0E2FA40F28C13C2F200031B6803F558
S31508001BB0FA63984207D340F28813C2F20003002260
S31508001BC01A7000F01FF808BD08B540F28813C2F273
S31508001BD0000301221A7000F0C7FA40F28C13C2F211
S31508001BE000031860FFF7D0FF08BD00BF704700BFAD
S31508001BF0704700BF08B5FFF7FBFFFCE708B500F024
S31508001C0051FD08BD10B500F06FFAB8B1FEF7CCFA71
S31508001C10A0B1FFF79DFD00F08DFA00F069FA20F0FB
S31508001C20604020F07F024EF60853CEF200031A6099
S31508001C3000F05EFA446800F037FDA04710BD00BF0B
S31508001C4070B5561EB6B24AB14C1E0E44451A14F863
S31508001C50013F2B55FFF7CCFFB442F8D170BD00BF4A
S31508001C6030B492B14B1C0331541EE4B201EB440468
S31508001C700021020F092A94BF3032373203F8012CAB
S31508001C80000103F8021BA342F3D130BC704700BF22
S31508001C9038B504460D46012807D942F2C870C0F681
S31508001CA000004FF4FC71FFF7A5FF40F21823C2F2BB
S31508001CB0000304EB440203EBC2035A7C1B7C9A42E2
S31508001CC020D040F21823C2F2000304EB440203EBCF
S31508001CD0C203DA681570597C01315974DA68013221
S31508001CE0DA605B689A420FD940F21823C2F2000301
S31508001CF06200111953F83110144403EBC403D96078
S31508001D00012038BD002038BD012038BD38B504464D
S31508001D100D46012807D942F2C870C0F6000040F205
S31508001D201A21FFF767FF40F21823C2F2000304EBFB
S31508001D30440203EBC2035B7CFBB140F21823C2F2F8
S31508001D40000303EBC2039A6812782A70597C01399A
S31508001D5059749A6801329A605B689A420FD940F2C0
S31508001D601823C2F200036200111953F83110144403
S31508001D7003EBC4039960012038BD002038BD01205B
S31508001D8038BD00BF10B540F21823C2F20003002088
S31508001D90987403F118025A61012183F82A10D8624F
S31508001DA040F21421C2F200010A604021197440F27F
S31508001DB08C21C2F200014C1C9C60DC6058741C60CB
S31508001DC001F140045C6008705AB340F21421C2F273
S31508001DD00001D86A0860402183F8281040F248219B
S31508001DE0C2F20001481C18625862002483F8294090
S31508001DF0986101F140035360927C0A7040F28C238B
S31508001E00C2F200031B78FF2B01D0FF2A06D142F24B
S31508001E10C870C0F600007A21FFF7ECFEFFF740F91C
S31508001E2010BD40F24823C2F20003FF221A70EEE703
S31508001E3008B50020FEF78CF908BD00BF2DE9F84368
S31508001E4007460C463F2906D942F2C870C0F600007C
S31508001E509921FFF7CFFE40F28C23C2F200031878CF
S31508001E602146FFF715FF012806D042F2C870C0F6D2
S31508001E7000009D21FFF7BEFE2646D4B1002440F29D
S31508001E808C25C2F2000542F2C878C0F600084FF069
S31508001E90A609FFF7ADFE2878395DFFF7F9FE012898
S31508001EA003D040464946FFF7A5FE0134A3B2B34224
S31508001EB0EFD3BDE8F88300BF10B50446FEF726FB4E
S31508001EC040F2D113C2F200031B7803BB40F2482349
S31508001ED0C2F20003187840F29011C2F20001FFF72F
S31508001EE015FF01283ED140F29013C2F200031B7879
S31508001EF0002B39D040F2D113C2F2000301221A7026
S31508001F0040F2D013C2F200030020187010BD40F250
S31508001F104823C2F2000340F2D012C2F2000211783E
S31508001F201878144B1944FFF7F1FE01281ED140F228
S31508001F30D013C2F200031A780132D2B21A7040F2F4
S31508001F409013C2F200031B78934211D12046094927
S31508001F50FFF776FE40F2D113C2F2000300221A7090
S31508001F60012010BD002010BD002010BD002010BDAE
S31508001F70002010BD910100202DE9F04383B040F206
S31508001F808C23C2F200031C78012C07D942F2C870D0
S31508001F90C0F6000040F23A21FFF72CFE40F2182363
S31508001FA0C2F2000304EB440403EBC4035B7C002B7E
S31508001FB03BD0402B34BF99464FF04009B9F1000F8A
S31508001FC023D040F2D413C2F200035C1E09F1FF3697
S31508001FD0F6B21E4440F28C25C2F2000542F2C877DA
S31508001FE0C0F6000740F2491828780DF10701FFF7F7
S31508001FF08DFE012803D038464146FFF7FBFD9DF8C4
S31508002000073004F8013FB442EED140F2D410C2F2D0
S3150800201000004FF480714A46FFF7D2F9012049467D
S31508002020FFF7E8FA0120FFF743FA03B0BDE8F083AB
S315080020302DE9F041012040F2D021C2F20001FFF75C
S315080020403BFB80B2F0B140F2D023C2F200035C1E23
S31508002050013886B21E4440F24825C2F2000542F213
S31508002060C877C0F600074FF4B778287814F8011F28
S31508002070FFF70EFE012803D038464146FFF7BAFDA2
S31508002080B442F2D10120FFF725FABDE8F08100BF7E
S3150800209038B54FF2E873C1F6FF731B684FF2EC725E
S315080020A0C1F6FF7214684FF2F072C1F6FF72126839
S315080020B0D0180AD0054D29460822FFF7D1FD20463B
S315080020C005F110010422FFF7CBFD38BD9A00002068
S315080020D008B500F05BF908BD08B500F065F908BD5C
S315080020E008B500F089F908BD08B500F071FA08BD11
S315080020F008B500F0C7FA08BD08B500F03DFA10B1FA
S3150800210000F09AFA08BD002008BD00BF4EF2100381
S31508002110CEF2000300221A6041F63F11C0F2010117
S3150800212059609A600521196040F21033C2F2000323
S315080021301A6070474EF21003CEF2000300221A60AE
S31508002140704700BF4EF21003CEF200031B6813F46B
S31508002150803F1FBF40F21033C2F200031A680132F3
S3150800216018BF1A60704700BF08B5FFF7EBFF40F2CB
S315080021701033C2F20003186808BD00BF4FF40053BD
S31508002180C4F202031A6942F080021A61704700BF5E
S31508002190F8B507460024254642F2F076C0F6000652
S315080021A0FFF726FDA359BB420ED8311949680B44DF
S315080021B09F4209D242F2F073C0F6000305EB4502CE
S315080021C003EB8203187AF8BD01350C349C2CE7D151
S315080021D0FF20F8BD2DE9F84380460068FFF7D8FFD1
S315080021E0FF285CD04FF40053C4F2020340F22312D6
S315080021F0C4F267525A6048F6AB12CCF6EF525A60F0
S315080022003422DA60DB6813F0010F04D0FFF7B6FF5B
S315080022100020BDE8F8834FF40053C4F202031A699C
S3150800222042F001021A61002508F104094FF400542E
S31508002230C4F20204D8F80030EF1859F80560B2B2B3
S31508002240EA52E36813F0010F05D0FFF7D1FCE36803
S3150800225013F0010FF9D1330C7B80E36813F0010FFB
S3150800226005D0FFF7C5FCE36813F0010FF9D13B6809
S31508002270B34204D10435B5F5007FDBD101E0002473
S3150800228000E001244FF40053C4F202031A6922F055
S3150800229001021A61FFF772FF2046BDE8F8830020A5
S315080022A0BDE8F88338B504460D4640F21433C2F249
S315080022B00003984209D04FF4C043C0F60003994280
S315080022C00BD0FFF787FF20B917E040F21854C2F287
S315080022D00004C5F3080393B903E040F21434C2F2CC
S315080022E0000423689D420CD0204640F8045B29462A
S315080022F04FF40072FFF7A4FC03E0002038BD00206D
S3150800230038BD204638BD00BF2DE9F04106460C46CB
S3150800231017461D464FEA51284FEA48280368B3F185
S31508002320FF3F06D140F8048B41464FF40072FFF791
S3150800233087FC3368434505D030464146FFF7B2FF70
S315080023400646D0B13368E41A3444043408F50078F4
S31508002350FFF74EFC331DE31AB3F5007F06D330466C
S315080023604146FFF79FFF064650B1041D17F8013B8B
S3150800237004F8013B013DEBD105E00020BDE8F08102
S315080023800020BDE8F0810120BDE8F08140F2185335
S31508002390C2F200034FF0FF321A6040F21433C2F261
S315080023A000031A60704700BF70B504460D4616460E
S315080023B0FFF7EEFEFF281BD0681E2044FFF7E8FE55
S315080023C0FF2817D0620A4FF4C043C0F60003B3EBE8
S315080023D0422F07BF40F21430C2F2000040F21850F4
S315080023E0C2F20000214632462B46FFF78DFF70BD2C
S315080023F0002070BD002070BD2DE9F84304460E4646
S31508002400FFF7C6FE0546701E2044FFF7C1FE0446C8
S31508002410FF2D18BFFF2800F0AB80854200F29F8091
S31508002420022D40F29F800F2800F29F804FF4005340
S31508002430C4F2020340F22312C4F267525A6048F605
S31508002440AB12CCF6EF525A603422DA60DB6813F02E
S31508002450010F04D0FFF792FE0020BDE8F8834FF481
S315080024600053C4F202031A6942F002021A6142F2E8
S31508002470F079C0F600094F460026FFF7B9FB3B7A0C
S31508002480AB4208D142F2F073C0F6000306EB4602EF
S3150800249053F8227005E001360C370D2EEDD14FF0BA
S315080024A0FF37C8460025FFF7A3FB98F80830A34274
S315080024B008D142F2F073C0F6000305EB450253F863
S315080024C0228006E0013508F10C080D2DEBD14FF0FE
S315080024D0FF384E460025FFF78BFB337AA34209D116
S315080024E042F2F073C0F6000305EB450203EB8203E4
S315080024F05B6804E001350C360D2DECD10023C7EBE3
S3150800250008084344C3F38F23E3B1013B9EB2013667
S31508002510B60200254FF40054C4F20204EB196361B5
S31508002520236943F040032361E36813F0010F05D0E4
S31508002530FFF75EFBE36813F0010FF9D105F5806537
S31508002540B542EBD14FF40053C4F202031A6922F0E4
S3150800255002021A61FFF712FE0120BDE8F883002087
S31508002560BDE8F8830020BDE8F8830020BDE8F883BD
S315080025700020BDE8F88300BF00B583B040F21433ED
S31508002580C2F200031B68B3F1FF3F08BF01201CD04D
S3150800259040F21433C2F2000399685A681144DA68A3
S315080025A011441A6911445A6911449A690A44D96945
S315080025B053185B4202AA42F8043D46F25010C0F690
S315080025C000000421FFF7F0FEFFE703B05DF804FB07
S315080025D046F20402C0F600024FF4C043C0F60003F8
S315080025E010681B68184446F20803C0F600031B6807
S315080025F0184446F20C03C0F600031B68184446F25A
S315080026001003C0F600031B68184446F21403C0F60C
S3150800261000031B68184446F21803C0F600031B683B
S31508002620184446F25013C0F600031B681844D0F14C
S31508002630010038BF0020704708B540F21433C2F2D3
S3150800264000031B68B3F1FF3F06D040F21430C2F214
S315080026500000FFF7BFFD88B140F21853C2F200032D
S315080026601B68B3F1FF3F0BD040F21850C2F20000CE
S31508002670FFF7B0FD003018BF012008BD002008BDD7
S31508002680012008BD4FF4C040C0F60000704700BFE7
S3150800269008B542F68C00C0F600003121FFF7AAFA09
S315080026A008BD00BF72B6704762B6704710B51549C7
S315080026B08D4640F20002C2F2000240F2ED03C2F279
S315080026C000039A4210D2131D0D4CE41A24F0030499
S315080026D004340023104642F6BC01C0F600015A58DD
S315080026E01A500433A342FAD1074808494FF00002AA
S315080026F08842B8BF40F8042BFADBFDF75DFD10BD34
S31508002700F00000205C090020F00000205A07002095
S315080027106D61696E2E630000120110010000004011
S31508002720501DAC6000010102030100000403090406
S315080027302603570069006E0055005300420020002A
S31508002740420075006C006B002000440065007600AE
S31508002750690063006500000009022000010100C04D
S31508002760320904000002FF00000407058102400048
S3150800277000070501024000001A034F0070006500BB
S315080027806E0042004C00540020005500730065009E
S31508002790720000002C03570069006E0055005300B4
S315080027A042002000420075006C006B0020004900C2
S315080027B06E007400650072006600610063006500C3
S315080027C04F70656E424C54002E2E2F2E2E2F2E2E15
S315080027D02F536F757263652F41524D434D335F53C7
S315080027E0544D333246312F7573622E630000000054
S315080027F000600008002000000300000000800008B8
S31508002800002000000400000000A0000800200000CE
S315080028100500000000C000080020000006000000B7
S3150800282000E0000800200000070000000000010882
S315080028300020000008000000002001080020000019
S315080028400900000000400108002000000A000000FE
S3150800285000600108002000000B000000008001084D
S31508002860002000000C00000000A001080020000065
S315080028700D00000000C00108002000000E00000046
S3150800288000E00108002000000F0000002E2E2F2E69
S315080028902E2F2E2E2F536F757263652F41524D437F
S315080028A04D335F53544D333246312F4743432F76CA
S311080028B06563746F72732E6300000000ED
S315080028BC5827000820000000D90300080104000866
S315080028CC710300087503000879030008C50300089E
S315080028DCC9030008B5040008C5040008D504000897
S315080028EC00000000400000009D1000084503000889
S315080028FC9D1000089D1000089D1000089D100008EA
S3150800290C9D1000089D100008610300086A2700083E
S3150800291C0900000018270008120000002C270008E0
S3150800292C04000000782700081A0000003027000869
S3150800293C26000000980000201C00000094270008C0
S3150800294C2C000000030100001C0353004500520034
S3150800295C31003200330034003500360037003800B9
S3150800296C390030001D0300089D1000089D10000852
S3150800297C9D1000089D1000089D1000089D10000869
S3150800298C250300089D1000089D1000089D100008DE
S3120800299C9D1000089D1000089D10000804FD
S70508000000F2
